:020000040000FA
:10000000C8420020E500000031120000D9000000C5
:1000100000000000000000000000000000000000E0
:10002000000000000000000000000000F1000000DF
:100030000000000000000000F3000000F5000000D8
:10004000F7000000F70000001D140000F70000009A
:10005000D9020000F7000000F7000000F7000000E0
:10006000F7000000F7000000F7000000F7000000B4
:10007000F7000000F7000000F7000000F7000000A4
:10008000F7000000F700000000000000F70000008B
:10009000F51100007D050000F7000000F7000000EA
:1000A000B3020000F7000000F7000000B1020000FA
:1000B000F7000000F7000000150D0000F700000039
:1000C0000448854600F0BAF800480047352400008F
:1000D000C046C046C84200207046694601F0ACFEEA
:1000E000FFF7FEFF0448804704480047FEE7FEE7AD
:1000F000FEE7FEE7FEE7FEE7A5150000C1000000F1
:1001000030B50B46014600202022012409E00D46AF
:10011000D5409D4205D31D469540491B2546954037
:1001200040191546521E002DF1DC30BD03460B432D
:100130009B0703D009E008C9121F08C0042AFAD29D
:1001400003E00B780370401C491C521EF9D2704723
:10015000D2B201E00270401C491EFBD2704700225F
:10016000F6E710B513460A4604461946FFF7F0FFB6
:10017000204610BD0321001D401E037812021A43C1
:10018000491EF9D510467047034603220870000A3D
:10019000491C521EFAD518467047F0B51FB40646E2
:1001A000002082B005464024019100901BE0019997
:1001B00022460F46304600F030F8049A059B801A1C
:1001C000994110D310461946224600F016F8361A07
:1001D0008F410197224601200021009F00F00DF879
:1001E00038184D4100902046641E0028DFDC019B3A
:1001F00000982946324607B0F0BD10B5202A04DB2E
:100200000146203A9140002010BD914020239C1AC5
:100210000346E3401943904010BD10B5202A04DB8B
:100220000846203AD040002110BD0B46D340D040B4
:100230002024A21A91400843194610BD064C0125FE
:10024000064E05E0E36807CC2B430C3C984710347E
:10025000B442F7D3FFF738FFA82F0000C82F0000E3
:100260007FB505460C466A462146284600F008FD43
:100270000098A0420FD16846C07900280BD168468B
:100280004079002807D168468079002803D1684664
:10029000007903280BD0029400216846C173417392
:1002A00081730321017302A9284600F049FD7FBD37
:1002B00070477047012806D1064989690122114318
:1002C000044A916105E00349896949084900014AE6
:1002D0009161704700240040002070470548C069C4
:1002E000FF2101310840002801D001207047002083
:1002F000FCE700000024004010B50446012C02D1A8
:100300001148036813E0022C03D10F484038C36B37
:100310000DE0032C03D10C484038836B07E0042C1C
:1003200003D109484038436B01E007480368180CC3
:10033000D94389B2884203D1D8B200F07FF802E0F5
:100340006B2000F07BF810BD40FBFF1F012806D199
:100350000649096BC2071143044A116305E00349CA
:10036000096B49004908014A1163704700240040A5
:100370000146064A106B130502469A4310461A4678
:100380000A401043014A10637047000000240040F7
:1003900030B502460B4600200F2424061440FF25EA
:1003A0002D066419002C09D06419002C08D064199A
:1003B000002C08D06419002C0BD107E00D4809E08F
:1003C0000C48001D06E00B48083003E009480C30DB
:1003D00000E000BF00BF00280BD092B20121914085
:1003E000002B03D004680C43046002E004688C43D3
:1003F000046030BD202400400146064A50680F23A7
:100400001B0402469A4310461A460A401043014A0A
:100410005060704700240040012806D10649496811
:1004200001221143044A516005E003494968490823
:100430004900014A51607047002400400146044AC7
:100440009068000A0002CAB21043014A90607047E7
:100450000024004010B504462068FFF7CDFF207946
:10046000FFF7DAFF10BD00000146064A10680723B7
:100470001B0202469A4310461A460A401043014A9C
:1004800010607047002400400146064A10680723A8
:100490001B0402469A4310461A460A401043014A7A
:1004A0001060704700240040012806D10749096800
:1004B00042061143054A116006E004490968012219
:1004C00052069143014A1160704700000024004029
:1004D0000146054A1068C008C0004A07520F104381
:1004E000014A1060704700000024004010B5044627
:1004F0002068FFF7EDFF6068FFF7B6FFA068FFF721
:10050000C3FF207BFFF7D0FF10BD0000012806D1FC
:100510000649496901221143044A516105E0034932
:10052000496949084900014A516170470024004067
:100530000146064A506907231B0202469A431046A9
:100540001A460A401043014A506170470024004097
:100550000320012189074860704700000146C80058
:10056000054BC218042310681840002801D0012050
:1005700070470020FCE700000404004010B507208D
:10058000FFF7ECFF012807D1072000F007F801284A
:1005900002D1072000F012F810BD00000146064805
:1005A000806A012212048A401040002801D00120F4
:1005B00070470020FCE700004004004001210904CE
:1005C0008140014A9162704740040040F8B50646F8
:1005D0000C461746032000F09FFF2102080E00F092
:1005E0009BFF2104080E00F097FFE0B200F094FF9B
:1005F000002505E0FF2000F08FFF7055681C85B2D4
:10060000BD42F7DB00F05EF8F8BDF7B584B07D21A0
:1006100049010698884202DD002007B0F0BD049829
:10062000029000200390059C069D002D0CD0200A0E
:10063000461C3002001BA84201D32F4601E03002C5
:10064000071B0120039001E00020039035E0062005
:1006500000F062FF022000F05FFF2102080E00F0B0
:100660005BFF2104080E00F057FFE0B200F054FFDA
:100670000020019009E002990878491C029100F0DD
:100680004BFF0198401C80B201900198B842F2D310
:10069000E419ED1B002D0CD0200A461C3002001B73
:1006A000A84201D32F4601E03002071B012003902E
:1006B00001E00020039000F005F803980028C6D15F
:1006C00000BFAAE710B500BF00F005F8C007C00FD3
:1006D0000028F9D110BD10B50A2001F017FD052042
:1006E00000F01AFFFF2000F017FF0446204610BD5F
:1006F0000146054A1068800880008A07920F10435F
:10070000014A10607047000000100040F7B5034632
:100710000D460021002207E0012696402E40002EC3
:1007200001D0114602E0521C102AF5D300BF102A56
:1007300000D1FEBD314FDE1BBB4211D008DC304E74
:100740009E19002E09D0402E08D0802E51D106E0EF
:10075000402E06D0802E4CD104E000BF00BF00BF69
:1007600000BF00BF254E4036B34203D0234E803633
:10077000B34202D10B2903D93CE00F2900D939E05B
:10078000032901D800200CE0042903D3072901D84C
:10079000012006E0082903D30B2901D8022000E03C
:1007A0000320164E803EB34200D1001D134E403E42
:1007B000B34200D10830114EB34200D10C300F4E7D
:1007C0004036B34200D110300C4E8036B34200D1D7
:1007D00014300C4E3469029E012E02D186403443FF
:1007E00004E0012686402746B7433C46054E346167
:1007F00000E000BF00BF00BF9BE70000C00C00404E
:1008000000F4FFBFC00D0040F0B502460D460023C6
:100810000027002407E00120A0402840002801D044
:10082000234602E0641C102CF5D300BF102C01D12C
:100830003846F0BD2E4E901BB24211D008DC2D4838
:100840001018002809D0402808D080284CD106E094
:10085000402806D0802847D104E000BF00BF00BF79
:1008600000BF00BF22484030824203D02048803081
:10087000824202D10B2B03D937E00F2B00D934E091
:10088000032B01D800210CE0042B03D3072B01D844
:10089000012106E0082B03D30B2B01D8022100E035
:1008A000032113488038824200D1091D1048403886
:1008B000824200D108310E48824200D10C310C48EE
:1008C0004030824200D1103109488030824200D14C
:1008D00014310948406901268E40304001268E407F
:1008E000B04200D1012700E000BF00BF3846A0E7BA
:1008F000C00C004000F4FFBFC00D0040F0B5024640
:100900000C460021002307E001269E402640002ED1
:1009100001D0194602E05B1C102BF5D300BF102B51
:1009200000D1F0BD2D4FD61BBA4211D008DC2C4EA1
:100930009619002E09D0402E08D0802E49D106E00D
:10094000402E06D0802E44D104E000BF00BF00BF7F
:1009500000BF00BF214E4036B24203D01F4E80364A
:10096000B24202D10B2903D934E00F2900D931E07A
:10097000032901D800200CE0042903D3072901D85A
:10098000012006E0082903D30B2901D8022000E04A
:100990000320124E803EB24200D1001D0F4E403E59
:1009A000B24200D108300D4EB24200D10C300B4E95
:1009B0004036B24200D11030084E8036B24200D1EB
:1009C0001430084E7569012686403540054E756124
:1009D00000E000BF00BF00BFA3E70000C00C004064
:1009E00000F4FFBFC00D0040F8B505460E4617469F
:1009F0001C4603223146284600F022F8314628469C
:100A000000F0A4F8224631462846FFF77FFE3A461A
:100A10003146284600F014F8C82001F077FB314633
:100A20002846FFF76BFF1E20002805DBC206D20E0A
:100A300001219140014A116000BFF8BD80E200E051
:100A4000F7B5034615460021002408E00126A6401C
:100A5000019F3E40002E01D0214602E0641C102C74
:100A6000F4D300BF102C00D1FEBD354FDE1BBB42BE
:100A700011D008DC334E9E19002E09D0402E08D02C
:100A8000802E58D106E0402E34D0802E53D132E053
:100A900000BF00BF00BF0F2900D94DE0032901D8D6
:100AA00000200CE0042903D3072901D8022006E026
:100AB000082903D30B2901D8042000E00620204E8A
:100AC000803EB34200D108301D4E403EB34200D1BB
:100AD00010301B4EB34200D118301B4EB2680326B3
:100AE00086401746B7433A462E4686403243164E56
:100AF000B26021E000BF0B2900D91DE0032901D815
:100B0000002006E0042903D3072901D8022000E0D1
:100B100004200B4E8036B34200D108300A4EF268F2
:100B2000032686401746B7433A462E468640324350
:100B3000054EF26000BF00BF00BF00BF94E7000099
:100B4000C00C004000F4FFBFC00D0040F0B50246ED
:100B50000D460020002407E00126A6402E40002E6E
:100B600001D0204602E0641C102CF5D300BF102CED
:100B700000D1F0BD3F4FD61BBA4234D008DC3E4E08
:100B80009619002E2CD0402E2BD0802E6ED129E02D
:100B9000402E02D0802E69D100E000BF0B2800D982
:100BA00065E0032801D8002106E0042803D30728C4
:100BB00001D8022100E004212E4E8036B24200D13D
:100BC00008318007800F2D4E736803268E401F4624
:100BD000B7433B4606468E403343284E736046E09B
:100BE00000BF00BF00BF234EC03EB24207D0214E1F
:100BF000803EB24203D01F4E403EB24202D10F2887
:100C000000D934E01B4EB24202D10B2800D92EE0AD
:100C1000032801D800210CE0042803D3072801D8B9
:100C2000022106E0082803D30B2801D8042100E0A4
:100C30000621104E803EB24200D108310D4E403E9A
:100C4000B24200D110310B4EB24200D118318007B0
:100C5000800F0A4E336803268E401F46B7433B463B
:100C600006468E403343054E336000E000BF00BFB0
:100C700000BF7EE7C00C004000F4FFBFC00D004085
:100C8000F0B504460025002307E001269E400E40F3
:100C90003546002D00D002E05B1C102BF5D300BFC1
:100CA000102B36D21D46116026680E403046E840B3
:100CB000012802D10126D67101E00026D6716668AE
:100CC0000E40EE403046012801D1967101E0002629
:100CD0009671A6680E40EE403046012801D156714B
:100CE00001E000265671E6686F00FE40B007800FF5
:100CF000002802D1002616710BE0012802D101263E
:100D0000167106E0022802D10226167101E00326C0
:100D10001671F0BD10B500F019FC40210648FFF730
:100D200073FD012806D140210348FFF7E7FD0120AC
:100D30000249087010BD0000C00C004000000020F7
:100D4000F0B502460B4600210024002500BF2DE02F
:100D500001268E4034461E6826403546A54224D1E1
:100D600010680646A6433046DE798E403043106058
:100D700050680646A64330469E798E403043506008
:100D800090680646A64330465E798E4030439060B8
:100D90004F000326BE403446D0680646A643304680
:100DA0001E794F00BE403043D060491C1029CFD37C
:100DB000F0BD02460020D3690B40002B01D001207A
:100DC00000E00020704781617047416170471FB5A6
:100DD0000446072202A9002000F0A1FA6846817BA0
:100DE0000170417B4170017B8170817AC170417AD1
:100DF0000171017A41710199009800F005FC012808
:100E000014D16846007A60716846407A207168465D
:100E1000807AE0706846007BA0706846407B607016
:100E20006846807B2070012004B010BD072202A913
:100E3000002000F074FA6846817B0170417B4170AC
:100E4000017B8170817AC170417A0171017A4171AF
:100E50000199009800F0D8FB012813D16846007A68
:100E600060716846407A20716846807AE070684612
:100E7000007BA0706846407B60706846807B207075
:100E80000120D1E70020CFE710B500F0F1FA0421EE
:100E90000C48FFF798FF012001F038F904210948B8
:100EA000FFF793FF042001F031F904210548FFF713
:100EB0008AFF042001F02AF904210248FFF785FF88
:100EC00010BD0000C00C004010B500F0D1FA0421A4
:100ED0000A48FFF77AFF012001F018F904210748BA
:100EE000FFF773FF042001F011F904210348FFF715
:100EF0006AFF042001F00AF910BD0000C00C004098
:100F000070B504211348FFF760FF00F0A1FA8024B8
:100F10001BE004210F48FFF758FF012001F0F6F80D
:100F200004210C48FFF745FF012803D12846204340
:100F3000054602E02846A043054604210548FFF780
:100F400042FF042001F0E2F86410002CE1D12846B1
:100F500070BD0000C00C004010B501210648FFF72D
:100F600017FA00220421054800F0A0F904210348E3
:100F7000FFF729FF10BD000007000001C00C004072
:100F800070B5054600F074FA80241BE02046284026
:100F9000002804D104211448FFF715FF03E00421C1
:100FA0001148FFF712FF012001F0B0F804210E48AC
:100FB000FFF70BFF042001F0A9F804210A48FFF70E
:100FC00002FF6410002CE1D1042001F09FF80421FD
:100FD0000548FFF7FAFE042001F098F804210248C2
:100FE000FFF7F1FE70BD0000C00C004010B5FFF728
:100FF000B3FF00F03DFA04210A48FFF7E6FE0421A2
:101000000848FFF7E2FE042001F080F804210548BB
:10101000FFF7D9FE042001F079F804210148FFF719
:10102000D2FE10BDC00C004010B500F021FA042122
:101030000C48FFF7C8FE04210A48FFF7C4FE04204D
:1010400001F064F804210748FFF7BFFE042001F017
:101050005DF804210348FFF7B8FE042001F056F8BC
:1010600010BD0000C00C00400148024908607047F4
:101070005A5A34120014014010B501210448FFF7F8
:1010800087F9062003494860FFF7EEFF10BD000016
:1010900005000001001401401CB500200090012053
:1010A000694608716846FFF7D5F90120FFF724F972
:1010B0001CBD00000A20054908600548008CC0B22C
:1010C0000449C861052001490860704700E00140FB
:1010D00000FBFF1F00F801401FB500240121194843
:1010E000FFF756F902211848FFF7BAF8042116480D
:1010F000FFF7B6F80120FFF709FA07200002FFF713
:1011000017FA052000F0DAFF0120FFF7D3F805E019
:1011100019200002844200D304E0641CFFF7DEF8CB
:101120000028F5D000BF012000900020019002901F
:101130000120694608736846FFF7D8F9034800F0B4
:1011400099FF1FBD07000001400D0040001BB700C4
:1011500010B50020FFF7CCFAFFF79EFFFFF7AAFFBC
:10116000FFF7BAFF10BD7FB506460D4614466A4626
:1011700029463046FFF784FD0098A84217D16846FB
:10118000C079012813D16846407901280FD1002C7D
:1011900003D168468079002809D1012C03D1684623
:1011A0008079012803D168460079002814D002957F
:1011B00001216846C1734173002C03D100206946A8
:1011C000887302E00120694688730020694608732D
:1011D00002A93046FFF7B4FD7FBD000004488069D6
:1011E000C007C00F002801D0012070470020FCE795
:1011F0000034014010B500F009F8012805D1FFF7CF
:10120000EDFF012801D100F00DF810BD0448406940
:1012100040210840002801D0012070470020FCE751
:1012200000340140402001494861704700340140CA
:101230007047000010B5002819DB1A4A03231B026F
:10124000D21883089B00D2588307DC0EFF23A340EB
:101250009A438B071B0E8407E40EA3401A43114BDD
:10126000032424021B198408A4001A5118E00E4A12
:1012700003071B0F083B9B089B00D2588307DC0E1B
:10128000FF23A3409A438B071B0E8407E40EA34061
:101290001A43054B0407240F083CA408A4001A5164
:1012A00010BD000000E100E01CED00E07FB5064647
:1012B0000D4614466A4629463046FFF7E1FC009881
:1012C000A84217D16846C079002813D1002C03D159
:1012D0006846407900280DD1012C03D16846407939
:1012E000012807D168468079002803D16846007933
:1012F000012813D0029500206946C873002C01D143
:10130000487302E0012069464873002168468173F2
:101310000121017302A93046FFF712FD7FBDF8B528
:1013200007460D4616460024FFF760FE6420FFF7CF
:1013300027FE3846FFF724FEFFF758FE6520FFF72B
:101340001FFE00BF06E0FFF7DBFD2855FFF79CFD01
:10135000601CC4B2701EA042F5DCFFF7D1FD285519
:10136000FFF7B2FDFFF760FEF8BDF8B507460D4682
:101370001646FFF73BFE6420FFF702FE3846FFF7F4
:10138000FFFD002404E0285DFFF7FAFD601CC4B2F5
:10139000B442F8DBFFF748FEF8BD00000146064AFC
:1013A0005068062302469A43104606220A4010431C
:1013B000014A50607047000000280040012806D113
:1013C0000649496801221143044A516005E0034976
:1013D000496849084900014A5160704700280040A7
:1013E000012806D10649096801221143044A116007
:1013F00005E00349096849084900014A116070473E
:101400000028004010B5FFF7A7FD01224021024847
:10141000FFF7A9FE10BD0000C00C00407047014658
:101420000869C007C00F002801D0012070470020C4
:10143000FCE70146086902221040002801D0012083
:1014400070470020FCE7014688697047416170479A
:1014500010B501210448FEF79BFF00220421034838
:10146000FFF781FE10BD000007000001C00C004026
:1014700010B501210448FEF78BFF00220421034828
:10148000FFF714FF10BD000007000001C00C004072
:10149000FFB585B004460D4616460E9F13A103C93D
:1014A000049103906846047145718671C7710F9964
:1014B00001726946109848720299019800F0A4F8E8
:1014C000012810D169461098087368460F99417336
:1014D00087730899C173067445748474072203A93D
:1014E0000020FFF742FF09B0F0BD0000000000003F
:1014F000010115001CB500216846017041700221F0
:1015000081700021C17040210171052269460B20C4
:10151000FFF72BFF1CBD000010B5044621460A480A
:10152000FFF794FF00BF0848FFF783FF0028FAD0B9
:1015300000BF0548FFF773FF0028FAD00248FFF705
:1015400082FF0446E0B210BD004C01401FB50024EC
:101550000120FEF7DBFF07200002FEF7E9FF032072
:1015600000F0ACFD0120FEF7A5FE05E01920000209
:10157000844200D304E0641CFEF7B0FE0028F5D0DE
:1015800000BF0120009000200190029001206946D8
:1015900008736846FEF7AAFF014800F06BFD1FBD07
:1015A000001BB70019200003024988600248034964
:1015B0000860704700ED00E000127A002000002073
:1015C00010B572B6FFF758FD0D4800F053FD0A2024
:1015D00000F074FDFFF7BCFD0120FFF701FF0620BE
:1015E000FFF7DCFE0020FFF7E9FEFEF7B1FF012167
:1015F0000448FEF7CDFEFFF737FD62B610BD0000D0
:1016000000127A0007000001F3B582B06E46357A09
:10161000EE17360F761937110A2677436E46307A61
:10162000C617360F361836113601861BBE19F1B2B1
:101630006E46757AEE17360F761937110A267743FC
:101640006E46707AC617360F361836113601861B6D
:10165000BE19F2B26E46B57AEE17360F761937110B
:101660000A2677436E46B07AC617360F36183611FB
:101670003601861BBE19F3B26E46F57AEE17360FA9
:10168000761937110A2677436E46F07AC617360F59
:10169000361836113601861BBE19F4B26E46357BFC
:1016A000EE17360F761937110A2677436E46307BD0
:1016B000C617360F361836113601861BBE19F6B21C
:1016C00001966E46757BEE17360F761936110A278E
:1016D0007E436F46787BC7173F0F3F183F113F018E
:1016E000C71BF619F6B20096632911DC14290FDB2B
:1016F0000C2A0DDC002A0BD01F2B09DC002B07D095
:10170000172C05DC01983B2802DC00983B2802DD01
:10171000002004B0F0BD0120FBE701468868C00747
:10172000C00F002801D0012070470020FCE7CA0547
:10173000D20D4261704700000FB410B503A9044BED
:10174000044A029800F02CF810BC08BC04B01847FA
:1017500009240000240000200FB410B504A9074B91
:1017600002AA039800F01CF8044602A9002000F029
:1017700051FA204610BC08BC04B01847151C0000E4
:1017800002E008C8121F08C1002AFAD1704770474A
:10179000002001E001C1121F002AFBD170470000A8
:1017A000FFB591B00F460546002606E025280AD071
:1017B000149A139990476D1C761C28780028F5D14F
:1017C000304615B0F0BD002400940121F34A029484
:1017D00000E004436D1C2B780846203B98401042E3
:1017E000F7D128782A280ED00222287801463039ED
:1017F000092915D800990A23594330394018144350
:101800006D1C0090F1E701CF0090002805DA01205F
:1018100040030443009840420090022004436D1CA2
:1018200028782E2815D10420044368786D1C2A28B6
:101830000AD101CF6D1C02900BE002990A2251439C
:10184000303940186D1C029028780146303909293A
:10185000F3D928786C2810D006DC4C281AD06828D8
:101860000ED06A2817D104E0742813D07A2812D138
:1018700010E00120400504430CE00121090501E0CE
:10188000032109050C436978814203D10120000539
:1018900024186D1C6D1C28786E281ED00CDC632863
:1018A00031D004DC00288BD0582811D1B2E0642854
:1018B0007BD069280CD178E073282DD004DC6F2808
:1018C00070D0702804D1A7E075286CD078286BD030
:1018D000149A13999047761C62E06002400F022828
:1018E00007D003280AD0042838680AD006603F1DB4
:1018F00056E03868F11706604160F8E738680680FE
:10190000F5E70670F3E738786946087400204874F4
:1019100004A80390012003E0386803900020C0432E
:101920003F1D61070FD5002101E00199491C029A72
:101930000191914213DA8142F7DB019A0399895CA4
:101940000029F2D10BE0002101E00199491C01912D
:101950008142FADB019A0399895C0029F5D101994A
:101960000098139A401A00902146149B00F03CF90D
:1019700001998019461807E0039803990078491CDB
:101980000391149A139990470198401E0190401CAE
:10199000F2D12146149B139A009800F015F986198C
:1019A0006D1C0AE741E033E034E00A200021049096
:1019B00005916002410F022905D001CFC21794465C
:1019C000032905D007E0FF1DFF08FF0003CF06E055
:1019D00000B2C2179446042902D140B2C1178C4606
:1019E00000226146944506DA0A46002140429141B0
:1019F0008C462D2102E0210504D52B216A46117663
:101A0000012103E0E10701D02021F7E7019155E032
:101A10000A200BE0102009E010200490002104208F
:101A2000044308200591029003E00820002105915D
:101A300004906002410F022905D001CF0022944694
:101A4000032906D006E0FF1DFF08FF0003CF8C46E8
:101A500003E080B2042900D1C0B200210191210726
:101A60002CD529780391702906D0049A1021059B62
:101A70004A401A4305D00EE040216A461176012102
:101A800008E06146014306D030216A461176039989
:101A9000517602210191049A0821059B4A401A437C
:101AA0000CD16146014301D1610707D530216A4657
:101AB0001176012101910299491E02912978582934
:101AC00004D037A103910FA90F910DE039A1F9E7D7
:101AD0006146059B049AFEF760FB039B8C469B5C6A
:101AE0000F9A521E0F92137061460143F0D10F9866
:101AF00007A9081A20300390600704D501200004CC
:101B00008443029801E0012002900399884201DD9C
:101B1000401A00E00020411802900198091800982E
:101B2000401A0090E00306D42146149B139A0098B3
:101B300000F05AF886190020049008E006A9085C15
:101B4000149A139990470498401C761C04900199AC
:101B50008842F3DBE0030CD52146149B139A0098CE
:101B600000F042F8861904E0149A30201399904747
:101B7000761C0299481E02900029F5DC08E00F98B7
:101B80000F990078491C0F91149A13999047761C6D
:101B90000399481E03900029F1DCFAE609280100A8
:101BA00030313233343536373839616263646566D3
:101BB0000000000030313233343536373839414295
:101BC0004344454600000000F8B5044600251E4683
:101BD0001746880404D405E039462020B0476D1C20
:101BE000641EF9D52846F8BDFFB50446002581B02E
:101BF0001E46C80301D5302700E02027880404D5FD
:101C000005E038460399B0476D1C641EF9D5284697
:101C100005B0F0BD0A68531C0B60107070470000DF
:101C200010B501208007FEF7A3FB0120FEF78EFB15
:101C300001231A4640210E48FEF7D6FE1E2000283A
:101C400005DBC206D20E012191400A4A116000BF95
:101C500000211E20FFF7EEFA1E20002806DBC20638
:101C6000D20E01219140034A803A116000BF10BD9D
:101C7000C00C004080E100E010B5FFF7C3FB10BDD1
:101C800010B5012400F0AEFC002800D1002410BDE6
:101C900010B500240C48FEF76DFA0C49884206D2B4
:101CA00000F091FB08490948FEF76EFA0124002C68
:101CB00008D02A2329221202FF2101310248801F65
:101CC00000F0D6FB10BD00002E00002001160424F9
:101CD00010B5012400F0A4FC002800D1002410BDA0
:101CE000F0B50446002B0CD125460E46002005E039
:101CF0002F783770761C6D1C471CB8B29042F7DB0A
:101D00000EE0012B0CD1A7187D1E0E46002005E029
:101D10002F783770761C6D1E471CB8B29042F7DBE7
:101D2000F0BD0000F7B584B0074616463B48006892
:101D3000039000253A48006802900020019039483D
:101D40000078002822D03848007800281ED1374873
:101D5000826928466D1C80003A5034484069441E10
:101D600033480068844211D331480068314909681A
:101D70004018A0420AD3102D08D20598854205D2FA
:101D800028466D1C80003C500120019026480078B8
:101D900000280CD00398864201D2039E07E00299E6
:101DA00003984018B04202D20299039846182DE0D9
:101DB0003068041FE007C00F002800D125E030681C
:101DC000441E1B480068001D84421DD3184800684B
:101DD000184909684018A04216D3102D14D2201FAC
:101DE00000F0BCF900280FD0059885420CD2022DD6
:101DF00006D10198002803D07868A04200D104E001
:101E000028466D1C80003C5000BF361D0299039887
:101E10004018B042CCD8284607B0F0BD0C000020D6
:101E2000100000201D0000201E0000208002002065
:101E30001400002018000020F0B58FB00E46354683
:101E40002C4620224D4907A8FEF770F94C48076838
:101E50004C48006806904C480078002809D14B4A4D
:101E60004BA14DA0FFF768FC53A0FFF765FC00BF36
:101E7000FEE752480078002809D0444A50A146A005
:101E8000FFF75AFC4CA0FFF757FC00BFFEE701200C
:101E90004A4908704DA0FFF74FFC47A0FFF74CFCE4
:101EA00000F0D2F84A49C86AFFF746FC42A0FFF7A3
:101EB00043FC2035BD4203D306983818A84202D20D
:101EC0000120444908702A463846069900F064F912
:101ED0004048007800284BD13D49086BFFF72CFCA7
:101EE00035A0FFF729FC3C4920680860606848601D
:101EF000A0688860E068C86020690861606948611E
:101F0000A0698861E069C8610846C068324A0A99D8
:101F10009268099B01930292039104902E484068B5
:101F200000902D48089B02682CA00799FFF704FC3D
:101F300021A0FFF701FC2848C069274A0E99926941
:101F40000D9B0193029203910490234840690090F5
:101F500021480C9B026921A00B99FFF7EDFB16A00D
:101F6000FFF7EAFB28A0FFF7E7FB13A0FFF7E4FB6E
:101F7000284600F099FA0FB0F0BD00006829000073
:101F80000C000020100000201C000020542900003C
:101F9000696E69745F6F6B0028257329206861730F
:101FA00020617373657274206661696C6564206179
:101FB000742025732E0000000D0A00001D00002073
:101FC000216F6E5F6661756C740000000000000098
:101FD000A82800001E000020800200202020257379
:101FE0003A2025303878202025733A20253038785B
:101FF000202025733A2025303878202025733A2078
:1020000025303878000000003D3D3D3D3D3D3D3DE3
:102010003D3D3D3D3D3D3D3D3D3D3D3D3D3D3D3DF0
:102020003D3D3D3D3D3D3D3D3D3D3D3D3D3D3D3DE0
:102030003D3D3D3D3D3D3D3D3D3D3D3D3D3D3D3DD0
:102040003D3D3D3D3D3D000010B50549054B064A6F
:1020500048680649FFF770FB05A0FFF76DFB10BD50
:10206000A8280000D0010020B0010020900100202D
:102070000D0A000010B504460C480068C0218843D2
:102080000A49086008460068C021084307490860FB
:1020900007492046FEF734F80649087008460078DC
:1020A0007D21C90048430449088010BD0024004038
:1020B00040420F0002000020040000200146114AA7
:1020C00012884A43104B5A6100229A611A461269DB
:1020D00001231A430C4B1A6100BF0B4A1069C20757
:1020E000D20F002A04D0012212040240002AF4D0A8
:1020F000054A126952085200034B1A6100229A6184
:10210000704700000400002000E000E00146114A92
:1021100012784A43104B5A6100229A611A4612699A
:1021200001231A430C4B1A6100BF0B4A1069C20706
:10213000D20F002A04D0012212040240002AF4D057
:10214000054A126952085200034B1A6100229A6133
:10215000704700000200002000E000E010B50146DA
:102160000B884A881F20C00210401F24E402A042AE
:1021700006D118400F242403A04201D1012010BD34
:10218000FF200002104047242402A04201D1012078
:10219000F5E70020F3E7000070B505460E4614464B
:1021A0001D48007800281CD01C480078002808D062
:1021B0001B4988692146FFF7BFFA1AA0FFF7BCFA4E
:1021C00007E01749C8692146FFF7B6FA15A0FFF7DF
:1021D000B3FAAC4201D22C4603E0A819A04200D2C7
:1021E000AC190F490869FFF7A7FA0EA0FFF7A4FA88
:1021F00008E021460CA02268FFF79EFA09A0FFF72D
:102200009BFA241DA819A042F3D80EA0FFF794FA58
:1022100004A0FFF791FA70BD1E0000201F000020EF
:10222000A82800000D0A00002020616464723A2092
:102230002530387820202020646174613A202530D0
:10224000387800003D3D3D3D3D3D3D3D3D3D3D3D02
:102250003D3D3D3D3D3D3D3D3D3D3D3D3D3D3D3DAE
:102260003D3D3D3D3D3D3D3D00000000FFB5FFB023
:10227000FFB085B007461C460021FFA8C1600121C0
:10228000890202A8FDF76BFF022101910026480296
:10229000844204DD00207FB07FB009B0F0BD00268D
:1022A0001FE00121890202A8FDF759FF2246FFA87D
:1022B000416902A8FEF78AF9A21E02A902312D483F
:1022C00000F0D8F905466846407A01026846007A6F
:1022D0000918A94203D10120FFA9C86003E0701CBE
:1022E000C6B2022EDDDB00BFFFA8C068012807D1FF
:1022F00000232246394602A8FFF7F2FC0120CAE774
:1023000000261FE00121890202A8FDF728FF2246CE
:10231000FFA8816902A8FEF759F9A21E02A902319D
:10232000144800F0A7F905466846407A010268465D
:10233000007A0918A94203D10120FFA9C86003E06F
:10234000701CC6B2022EDDDB00BFFFA8C0680128EA
:102350000DD100232246394602A8FFF7C1FC2246D0
:10236000FFA8416902A8FEF750F9012093E7002079
:1023700091E70000FFFF0000F8B506460F4614463F
:102380001D46012000902A463946304600F01CF8D0
:10239000002807D12A463946304600F015F80028B3
:1023A00000D100902A462146304600F00DF8002862
:1023B00007D12A462146304600F006F8002800D111
:1023C00000900098F8BD704770B5FFB0FFB082B0C4
:1023D00005460E46144601208002844204DD00209A
:1023E0007FB07FB002B070BD224631462846FEF76E
:1023F0000CF9224631466846FEF7E8F8224669465F
:10240000284600F021F9EBE770B504460E46E5B228
:1024100029460548FFF78BF900BF0348FFF77DF910
:102420000028FAD0284670BD0020014010B5FFF703
:1024300023FC10BDFFF7C4F8FFF7F8FF00F09CF88D
:1024400000F07EF8FFF7ECFBFEF70EFE0BE006480F
:102450000078012807D1002003490870FEF704FE28
:102460000248FEF7B4FCF2E700000020060000205E
:10247000FFB581B004460F461D46AA1EA11C09489F
:1024800000F0F8F806462670301260702B46394688
:102490002046039AFFF770FF002801D105B0F0BD78
:1024A0000120FBE7FFFF000070B592B00646002553
:1024B000402102A8FDF753FE3246102102A8FFF783
:1024C00031FC0546002410E0A10002AB5A58E1009F
:1024D0006118134BC81813A1FFF73EF92021E00043
:1024E000201808300E4A1154641CAC42ECD3002D65
:1024F0000DD00B48E9006B180C4900900CA2086A3B
:102500000D49FFF719F90DA0FFF716F906E0074985
:10251000486AFFF711F909A0FFF70EF912B070BD74
:10252000F00100202530386C78000000A828000059
:102530002E61786600000000900100200D0A000066
:102540000EB5FEF7D7FF0A48FEF741FC00280ED172
:102550000848C1798079074A5279064B0092029166
:1025600001901A79D97898780123FEF791FF0EBD72
:1025700006000020E600002010B596B02C210BA824
:10258000FDF7EDFD2C216846FDF7E9FD01242A2227
:1025900021020BA8FEF71AF80BA80230FDF7EAFD9E
:1025A0000F49884200D10FE02A22292109026846FA
:1025B000FEF70CF800A80230FDF7DCFD0849884260
:1025C00001D1012400E00024002C02D1FFF758FBC8
:1025D00001E0FFF77DFBFFF75BFB16B010BD0000CD
:1025E0000116042410B50C490C48FDF7CDFD0A492D
:1025F000091D0A48FDF7C8FD202107480830FDF7EE
:10260000AEFD2A2329221202FF2101310248801E39
:10261000FFF72EFF10BD00002A0000200116042441
:1026200010B52A2329221202FF2101310548FFF7A4
:102630001DFE002803D1FFF7D5FF002010BD0120AB
:10264000FCE700002800002070B503460C4600217E
:10265000002000BF07E05D5C665CB54201D0002051
:1026600003E04D1CA9B29142F5DB00BF914200D1BD
:10267000012070BDF0B5034614461D12DEB208E01D
:102680000A78491C72400648805C68400646054846
:10269000855C2046641E0028F2D128023043F0BD3C
:1026A000A8260000A827000000C1814001C0804189
:1026B00001C0804100C1814001C0804100C1814012
:1026C00000C1814001C0804101C0804100C1814002
:1026D00000C1814001C0804100C1814001C08041F2
:1026E00001C0804100C1814001C0804100C18140E2
:1026F00000C1814001C0804100C1814001C08041D2
:1027000001C0804100C1814000C1814001C08041C1
:1027100001C0804100C1814001C0804100C18140B1
:1027200000C1814001C0804101C0804100C18140A1
:1027300000C1814001C0804100C1814001C0804191
:1027400001C0804100C1814000C1814001C0804181
:1027500001C0804100C1814001C0804100C1814071
:1027600000C1814001C0804100C1814001C0804161
:1027700001C0804100C1814001C0804100C1814051
:1027800000C1814001C0804101C0804100C1814041
:1027900000C1814001C0804100C1814001C0804131
:1027A00001C0804100C1814000C0C101C30302C219
:1027B000C60607C705C5C404CC0C0DCD0FCFCE0E81
:1027C0000ACACB0BC90908C8D81819D91BDBDA1AF1
:1027D0001EDEDF1FDD1D1CDC14D4D515D71716D661
:1027E000D21213D311D1D010F03031F133F3F232D1
:1027F00036F6F737F53534F43CFCFD3DFF3F3EFE41
:10280000FA3A3BFB39F9F83828E8E929EB2B2AEAB0
:10281000EE2E2FEF2DEDEC2CE42425E527E7E62620
:1028200022E2E323E12120E0A06061A163A3A26290
:1028300066A6A767A56564A46CACAD6DAF6F6EAE00
:10284000AA6A6BAB69A9A86878B8B979BB7B7ABA70
:10285000BE7E7FBF7DBDBC7CB47475B577B7B676E0
:1028600072B2B373B17170B0509091519353529250
:1028700096565797559594549C5C5D9D5F9F9E5EC0
:102880005A9A9B5B99595898884849894B8B8A4A30
:102890004E8E8F4F8D4D4C8C4484854587474686A0
:1028A0008242438341818040482B0000382A000047
:1028B000BC2B0000A02B0000A4290000CC290000A4
:1028C000482F0000642F0000682A0000D42B00006D
:1028D000042B0000E42A0000F4290000702C000002
:1028E000B82C0000E82B0000A02D0000682D00008F
:1028F000C82E0000742E0000202E0000482E00007C
:10290000242F0000002F0000982E0000F02C000063
:10291000202B0000482C0000182D0000782B000010
:10292000802F0000FC2D0000942C0000242C0000BF
:10293000442D0000D82D0000C42A0000A82A000061
:10294000636D5F6261636B74726163655F61737312
:1029500065727400636D5F6261636B74726163655D
:102960005F6661756C740000882900008C29000086
:102970009029000094290000A02900009C29000053
:1029800098290000342A00005230200052312000E3
:102990005232200052332000504320004C5220007D
:1029A000523132003D3D3D3D3D3D3D3D3D3D3D20B3
:1029B000CFDFB3CCB6D1D5BBD0C5CFA2203D3D3DF6
:1029C0003D3D3D3D3D3D3D3D000000003D3D3D3D2B
:1029D0003D3D3D3D3D3D3D3D20D6F7B6D1D5BBD03B
:1029E000C5CFA2203D3D3D3D3D3D3D3D3D3D3D3DB5
:1029F000000000003D3D3D3D3D3D3D3D3D3D3D3DFB
:102A00003D3D3D3D3D3D3D3D3D3D3D3D3D20BCC40D
:102A1000B4E6C6F7D0C5CFA2203D3D3D3D3D3D3D8E
:102A20003D3D3D3D3D3D3D3D3D3D3D3D3D3D3D3DD6
:102A30003D3D000050535200B9CCBCFEC3FBB3C6B1
:102A4000A3BA2573A3ACD3B2BCFEB0E6B1BEBAC57F
:102A5000A3BA2573A3ACC8EDBCFEB0E6B1BEBAC53F
:102A6000A3BA257300000000B2E9BFB4B8FCB6E019
:102A7000BAAFCAFDB5F7D3C3D5BBD0C5CFA2A3ACFF
:102A8000C7EBD4CBD0D0A3BA61646472326C696EE8
:102A900065202D652025732573202D61202D66204E
:102AA000252E2A7300000000B7A2C9FAD7DCCFDFB9
:102AB000B4EDCEF3B5C4B5D8D6B7A3BA25303878BF
:102AC00000000000B7A2C9FAB4E6B4A2C6F7B9DCA8
:102AD000C0EDB4EDCEF3B5C4B5D8D6B7A3BA2530A2
:102AE00038780000D4DAD6D0B6CFBBF2C2E3BBFA56
:102AF000BBB7BEB3CFC2B7A2C9FAB4EDCEF3D2EC26
:102B0000B3A30000D4DACFDFB3CC28257329D6D005
:102B1000B7A2C9FAB4EDCEF3D2ECB3A30000000023
:102B2000B7A2C9FAD3C3B7A8B4EDCEF3A3ACD4AD62
:102B3000D2F2A3BACAD4CDBCC7D0BBBBB5BD20416D
:102B4000524D20D7B4CCAC00B4EDCEF3A3BACEDE58
:102B5000B7A8BBF1C8A1D6F7D5BBD0C5CFA2A3AC4F
:102B6000C7EBBCECB2E9D6F7D5BBB5C4CFE0B9D85A
:102B7000C5E4D6C300000000B7A2C9FAD3C3B7A802
:102B8000B4EDCEF3A3ACD4ADD2F2A3BAC6F3CDBCB0
:102B9000D6B4D0D0B7C7B6D4C6EBB7C3CECA000040
:102BA000D4DAD6D0B6CFBBF2C2E3BBFABBB7BEB362
:102BB000CFC2B7A2C9FAB6CFD1D40000D4DACFDFE2
:102BC000B3CC28257329D6D0B7A2C9FAB6CFD1D4B1
:102BD00000000000BBF1C8A1BAAFCAFDB5F7D3C36E
:102BE000D5BBCAA7B0DC0000B7A2C9FAB4E6B4A24C
:102BF000C6F7B9DCC0EDB4EDCEF3A3ACD4ADD2F2E0
:102C0000A3BAC6F3CDBCB4D3B2BBD4CAD0EDB7C35C
:102C1000CECAB5C4C7F8D3F2B6C1A1A2D0B4CAFD1A
:102C2000BEDD0000B7A2C9FAB5F7CAD4B4EDCEF341
:102C3000A3ACD4ADD2F2A3BACAFDBEDDBCE0B2E211
:102C4000B5E3C6A5C5E40000B7A2C9FAD3C3B7A8C7
:102C5000B4EDCEF3A3ACD4ADD2F2A3BACEDED0A7FE
:102C6000B5C4D2ECB3A3B7B5BBD8C2EB000000002B
:102C7000B7A2C9FAD3B2B4EDCEF3A3ACD4ADD2F2BD
:102C8000A3BAC8A1D6D0B6CFCFF2C1BFCAB1B3F6EE
:102C9000B4ED0000B7A2C9FAB5F7CAD4B4EDCEF3CB
:102CA000A3ACD4ADD2F2A3BAD6B4D0D020424B500C
:102CB0005420D6B8C1EE0000B7A2C9FAB4E6B4A257
:102CC000C6F7B9DCC0EDB4EDCEF3A3ACD4ADD2F20F
:102CD000A3BAC6F3CDBCB4D3B2BBD4CAD0EDB7C38C
:102CE000CECAB5C4C7F8D3F2C8A1D6B8C1EE0000A9
:102CF000B7A2C9FAD3C3B7A8B4EDCEF3A3ACD4AD91
:102D0000D2F2A3BAC6F3CDBCD6B4D0D0CEB4B6A856
:102D1000D2E5D6B8C1EE0000B7A2C9FAD3C3B7A8AE
:102D2000B4EDCEF3A3ACD4ADD2F2A3BAC6F3CDBC0E
:102D3000D6B4D0D0D0ADB4A6C0EDC6F7D6B8C1EEEB
:102D400000000000B7A2C9FAB5F7CAD4B4EDCEF3BB
:102D5000A3ACD4ADD2F2A3BAB7A2C9FACFF2C1BF25
:102D6000B2B6BBF100000000B7A2C9FAB4E6B4A243
:102D7000C6F7B9DCC0EDB4EDCEF3A3ACD4ADD2F25E
:102D8000A3BAC8EBD5BBCAB1C6F3CDBCB7C3CECAD4
:102D9000B2BBB1BBD4CAD0EDB5C4C7F8D3F2000002
:102DA000B7A2C9FAB4E6B4A2C6F7B9DCC0EDB4ED77
:102DB000CEF3A3ACD4ADD2F2A3BAB3F6D5BBCAB1AD
:102DC000C6F3CDBCB7C3CECAB2BBB1BBD4CAD0ED7B
:102DD000B5C4C7F8D3F20000B7A2C9FAB5F7CAD490
:102DE000B4EDCEF3A3ACD4ADD2F2A3BACDE2B2BF70
:102DF000B5F7CAD4C7EBC7F300000000B7A2C9FA01
:102E0000B5F7CAD4B4EDCEF3A3ACD4ADD2F2A3BA25
:102E10004E56494320CDA3BBFAC7EBC7F3000000D1
:102E2000B7A2C9FAD7DCCFDFB4EDCEF3A3ACD4ADF3
:102E3000D2F2A3BABEABC8B7B5C4CAFDBEDDD7DCFB
:102E4000CFDFB4EDCEF30000B7A2C9FAD7DCCFDFF5
:102E5000B4EDCEF3A3ACD4ADD2F2A3BAB2BBBEAB49
:102E6000C8B7B5C4CAFDBEDDD7DCCFDFB4EDCEF345
:102E700000000000B7A2C9FAD7DCCFDFB4EDCEF373
:102E8000A3ACD4ADD2F2A3BAD6B8C1EED7DCCFDFB3
:102E9000B4EDCEF300000000B7A2C9FAD7DCCFDF53
:102EA000B4EDCEF3A3ACD4ADD2F2A3BAB6E8D0D48D
:102EB000B1A3B4E6B8A1B5E3D7B4CCACCAB1B7A25C
:102EC000C9FAB4EDCEF30000B7A2C9FAB4E6B4A2D1
:102ED000C6F7B9DCC0EDB4EDCEF3A3ACD4ADD2F2FD
:102EE000A3BAB6E8D0D4B1A3B4E6B8A1B5E3D7B4D9
:102EF000CCACCAB1B7A2C9FAB4EDCEF30000000061
:102F0000B7A2C9FAD7DCCFDFB4EDCEF3A3ACD4AD12
:102F1000D2F2A3BAC8EBD5BBCAB1B7A2C9FAB4ED15
:102F2000CEF30000B7A2C9FAD7DCCFDFB4EDCEF301
:102F3000A3ACD4ADD2F2A3BAB3F6D5BBCAB1B7A293
:102F4000C9FAB4EDCEF30000B4EDCEF3A3BACFDFEF
:102F5000B3CCD5BB282530387829B7A2C9FAD2E737
:102F6000B3F60000B4EDCEF3A3BAD6F7D5BB28254F
:102F700030387829B7A2C9FAD2E7B3F600000000CA
:102F8000B7A2C9FAD3C3B7A8B4EDCEF3A3ACD4ADFE
:102F9000D2F2A3BAC6F3CDBCD6B4D0D0B3FD2030A4
:102FA00020B2D9D7F7000000C82F00000000002091
:102FB0002800000080170000F02F000028000020EB
:102FC000A04200009017000000000000000018015F
:102FD00001000000000000000000000000000000F0
:102FE000000000000000000000127A000000000055
:04000005000000C136
:00000001FF
